:100000000C94EF050C9437060C9437060C943706C5
:100010000C9437060C9437060C9437060C9437066C
:100020000C9437060C9437060C9437060C94FD1785
:100030000C9437060C9465260C9437060C943706FE
:100040000C9437060C9437060C9437060C94BE2695
:100050000C9437060C9437060C9437060C9437062C
:100060000C9437060C9437060C9437060C9437061C
:100070000C94370663168A1682178A168217D616CC
:10008000F916821750175F17981C981CD01CD01CAB
:100090004B1D7F1D761F761F961D761F271D271D62
:1000A000301F761F451F631F041607090B0A1D1B0F
:1000B00006196405141A08151C171E1F2021232277
:1000C0002E26242D25273012182F0C13280F0D341F
:1000D0000E333136381110372B2C352A5829787BBE
:1000E00079397A504F5152808063685680668053C8
:1000F0000201035558805780805462595A5B5C5DF9
:100100005E5F8060617475673E3F403C414277446A
:1001100076460047804365453248494A4B4C3D4D41
:100120003B4E3A7D7E7C7F73413A2425583A41709C
:10013000706C69616E6365284D65646961206B65EB
:100140007973290A004D3A2425583A4B656E736934
:100150006E67746F6E0A004D3A2425583A457874DC
:10016000656E6465640A004D3A2425583A4C6F6701
:1001700069746563682D457874656E6465640A000A
:100180004D3A2425583A4C6F6769746563680A00D4
:100190004D3A2425583A4D6163616C6C792D326279
:1001A000746E0A004D3A2425583A4B656E73696E99
:1001B00067746F6E204578740A004D3A2425583ACA
:1001C0004558543A205B253032582025303258208B
:1001D00025303258202530325820253032582025FD
:1001E000303258202530325820253032585D206377
:1001F00070693D25642062746E3D2564206C656ED7
:100200003D25640A004D3A2425583A436C617373C6
:10021000696332203230306370690A004D3A242518
:10022000583A436C617373696331203130306370C5
:10023000690A004D3A2425583A53657475702E208A
:1002400052333A253034580A004D3A2425583A4E54
:100250006F7420666F756E640A004B3A2425583A15
:100260004C61796F75743A2025730A004B3A242546
:10027000583A53657475702E2052333A25303458ED
:100280000A004B3A2425583A4E6F7420666F756EFB
:10029000640A00523A2425583A4D6F766520746FEF
:1002A000202425582E2052333A253034580A005243
:1002B0003A2425583A4661696C20746F206D6F7638
:1002C000650A00523A2425583A4E6F2066726565D9
:1002D00020616464726573730A00523A2425583AA7
:1002E000466F756E642E2052333A253034580A001A
:1002F0006D3A556E6B6E6F776E3A20253032580A24
:10030000006D3A2425583A2530345820005B2042AD
:100310003A2530325820583A256428256429205936
:100320003A25642825642920563A2564205D0A0070
:100330005D20002530325820004D3A2425583A25BA
:100340003032583A5B20000A0025583A253032589E
:100350002025583A253032580A002D2D2D2D2D2DCF
:100360002D2D2D0A00413A482020613A680A000AE2
:100370005461626C653A0A004B3A2425583A25309C
:1003800032583A2530345820005D0A002530325862
:100390002000553A2425583A253032583A5B20003F
:1003A0000A002425582052333A253034580A000ACE
:1003B0005363616E3A0A007300530052000A4C6F97
:1003C0006F702073746172742E0A000A55534220B4
:1003D000636F6E666967757265642E0A000A544D14
:1003E0004B3A6334366437622F4C5546413A643693
:1003F000613764660A002E03410044004200200079
:100400006B006500790062006F006100720064009B
:10041000200063006F006E007600650072007400BB
:100420006500720000000E0374002E006D002E00A7
:100430006B002E00000004030904090254000301AC
:1004400000A032090400000103010100092111018B
:1004500000012240000705810308000A0904010089
:100460000103010200092111010001227F0007059B
:1004700082030800010904020001030000000921B1
:10048000110100012222000705830320000112014F
:10049000100100000008EDFEDB0A0101010200016D
:1004A0000631FF0974A1010975150026FF0095208A
:1004B000750881020976150026FF009520750891C0
:1004C00002C005010902A1010901A1008501050978
:1004D00019012908150025019508750181020501FA
:1004E000093009311581257F950275088106093883
:1004F0001581257F950175088106050C0A380215BE
:1005000081257F950175088106C0C005010980A17C
:100510000185021601002637001A81002AB70075EE
:100520001095018100C0050C0901A1018503160188
:1005300000269C021A01002A9C0275109501810078
:10054000C005010906A101050719E029E7150025E5
:100550000195087501810295017508810105081949
:100560000129059505750191029501750391010514
:1005700007190029FF150026FF0095067508810060
:10058000C0636F6E73756D65723A20253034580AFA
:100590000073797374656D3A20253034580A000A67
:1005A000002530325820006B6579626F6172643AC1
:1005B00020004C45443A20253032580A0025583A4C
:1005C0002530386225730A000A2020303132333456
:1005D0003536370A00290A002575002F00257500D9
:1005E0005D280025640020002564002000256400AB
:1005F00020002564007C0025303258006D6F757333
:10060000656B6579205B62746E7C7820792076203A
:10061000685D287265702F61636C293A205B006DFC
:100620006B5F776865656C5F74696D655F746F5F3C
:100630006D6178203D2025640A006D6B5F776865E9
:10064000656C5F6D61785F7370656564203D202522
:10065000640A006D6B5F74696D655F746F5F6D61D7
:1006600078203D2025640A006D6B5F6D61785F73B3
:1006700070656564203D2025640A006D6B5F696EBE
:1006800074657276616C203D2025640A006D6B5F95
:1006900064656C6179203D2025640A006D6B5F778D
:1006A0006865656C5F74696D655F746F5F6D6178B7
:1006B000203D2025640A006D6B5F776865656C5F7F
:1006C0006D61785F7370656564203D2025640A0064
:1006D0006D6B5F74696D655F746F5F6D6178203DF0
:1006E0002025640A006D6B5F6D61785F73706565CE
:1006F00064203D2025640A006D6B5F696E7465722D
:1007000076616C203D2025640A006D6B5F64656C2A
:100710006179203D2025640A000A00257500363ADB
:1007200020776865656C5F74696D655F746F5F6D78
:1007300061783A20000A00257500353A207768650F
:10074000656C5F6D61785F73706565643A20000A5F
:1007500000257500343A2074696D655F746F5F6DB4
:1007600061783A20000A00257500333A206D6178DF
:100770005F73706565643A20000A00257500323A9F
:1007800020696E74657276616C286D73293A200059
:100790000A00257500313A2064656C6179282A3198
:1007A000306D73293A20000A092D2056616C756559
:1007B00073202D0A004D3E004D25643E20003F0071
:1007C0007365742064656661756C740A00433E202D
:1007D0000077686572652064656C74613A206375A2
:1007E00072736F723D25642C20776865656C3D25BA
:1007F000640A53656520687474703A2F2F656E2EF5
:1008000077696B6970656469612E6F72672F7769AC
:100810006B692F4D6F7573655F6B6579730A000A9D
:10082000092D204D6F7573656B6579202D0A455331
:10083000432F713A09717569740A313A0964656C1C
:100840006179282A31306D73290A323A09696E7448
:10085000657276616C286D73290A333A096D617887
:100860005F73706565640A343A0974696D655F7415
:100870006F5F6D61780A353A09776865656C5F6D01
:1008800061785F73706565640A363A0977686565F3
:100890006C5F74696D655F746F5F6D61780A0A7073
:1008A0003A097072696E742076616C7565730A64BA
:1008B0003A097365742064656661756C74730A75B2
:1008C000703A092B310A646F776E3A092D310A703C
:1008D0006775703A092B31300A7067646F776E3A2A
:1008E000092D31300A0A7370656564203D20646506
:1008F0006C7461202A206D61785F73706565642077
:100900002A2028726570656174202F2074696D65D6
:100910005F746F5F6D6178290A003F004D3E2000D3
:10092000433E20004C25640A000A092D20436F6EC7
:10093000736F6C65202D0A4553432F713A09717509
:1009400069740A6D3A096D6F7573656B65790A0094
:100950000A092D204D61676963202D0A643A0964F4
:10096000656275670A783A096465627567206D612A
:10097000747269780A6B3A096465627567206B6501
:1009800079626F6172640A6D3A0964656275672005
:100990006D6F7573650A763A0976657273696F6E65
:1009A0000A733A097374617475730A633A09636F61
:1009B0006E736F6C65206D6F64650A302D343A0973
:1009C0006C61796572302D34284631302D463429DA
:1009D0000A506175733A09626F6F746C6F61646578
:1009E000720A003F0074696D65725F7265616433FD
:1009F0003228293A202530346C580A006B65796218
:100A00006F6172645F69646C653A2025580A006BF7
:100A10006579626F6172645F70726F746F636F6C1F
:100A20003A2025580A00686F73745F6B6579626FAE
:100A30006172645F6C65647328293A2025580A0046
:100A40000A092D20537461747573202D0A004743E1
:100A5000433A20352E342E30204156522D4C4942F7
:100A6000433A20322E302E30204156525F415243BD
:100A7000483A2061767233350A004F5054494F4E40
:100A8000533A204C554641204D4F5553454B4559FF
:100A90002045585452414B455920434F4E534F4CDB
:100AA0004520434F4D4D414E44204B45594D4150FB
:100AB0005F53454354494F4E20343039360A004283
:100AC00055494C443A206334366437622028313922
:100AD0003A34303A3231204D61792033302032308F
:100AE0003232290A005649443A2030784645454476
:100AF00028742E6D2E6B2E29205049443A203078D0
:100B00003041444228414442206B6579626F6172F2
:100B10006420636F6E766572746572292056455243
:100B20003A203078303130310A00444553433A207E
:100B3000636F6E7665727420414442206B65796202
:100B40006F61726420746F205553420A000A092DA8
:100B50002056657273696F6E202D0A000A6D6F75DD
:100B600073653A206F66660A000A6D6F7573653AA1
:100B7000206F6E0A000A6B6579626F6172643A20B9
:100B80006F66660A000A6B6579626F6172643A206B
:100B90006F6E0A000A6D61747269783A206F66663A
:100BA0000A000A6D61747269783A206F6E0A000A51
:100BB00064656275673A206F6E0A000A6465627543
:100BC000673A206F66660A000A0A626F6F746C6F7C
:100BD000616465722E2E2E2000433E2000001124F9
:100BE0001FBECFEFD4E0DEBFCDBF04B603FE28C0EA
:100BF0008091B3039091B403A091B503B091B60373
:100C00008730904BA740B04BD9F41092B3031092A9
:100C1000B4031092B5031092B60314BE0FB6F89445
:100C2000A8958091600088618093600010926000B8
:100C30000FBE1092010810920008E0E0F8E3099559
:100C400011E0A0E0B1E0E2E8FEE502C005900D92FF
:100C5000A435B107D9F723E0A4E5B1E001C01D92A6
:100C6000A33BB207E1F70E947C130C943F2F0C9436
:100C70000000FF93EF93E0915401F09155013097FC
:100C800009F00995EF91FF910895FC01859180305D
:100C900011F0EFDFFBCF0895FF27E0E230E247FFDE
:100CA0000CC0419597FF09C0EDE260957095809565
:100CB0009095611D711D811D911D27FF02C0219519
:100CC00030E350E2AA27660F771F881F991FAA1FDB
:100CD000A41710F0A41B63955A95A9F7AA3008F041
:100CE000A95FA05DAF93F39561157105810591052D
:100CF00041F7ED3211F4EF93F395F21718F43F93A7
:100D0000F395FBCF8F91B5DFFA95E1F70895E9915F
:100D1000F9918591803021F0853219F0AADFF9CF61
:100D2000089520E0E89455915532C1F3503311F401
:100D3000689455915A3348F4505390F3220F022E81
:100D4000220F220F200D250FF4CF0EF4219589914B
:100D50009991533619F3533729F1533559F1BC01A1
:100D600088279927E8945C3621F4899199916894B1
:100D70005591543639F446EF7EF077FF0DC08FEF72
:100D80009FEF0AC055374AE039F0583540E121F06D
:100D9000523642E009F00895FF93EF937DDFEF9123
:100DA000FF91B7CFFF93EF93FC0181918030B9F3AE
:100DB00060DFFBCFFF93EF9368DFF1CFDF93CF933B
:100DC000CDB7DEB72596A3DFCF91DF910895282F09
:100DD0002770E82FE695E695E695EF70F0E0EC5683
:100DE000FE4F87FF0AC081E090E001C0880F2A957E
:100DF000EAF780959081892308C081E090E001C0E6
:100E0000880F2A95EAF79081892B8083089589318C
:100E100091F1C0F48D3079F150F4873061F120F414
:100E20008450823060F527C0893049F524C0843170
:100E300011F128F48131F9F08231F9F020C08831C4
:100E4000E0F01DC0823CC9F058F48D31A1F018F4D7
:100E50008A3199F014C08E3181F0813C81F40BC04D
:100E6000873C49F028F4843C31F0853C31F007C0E0
:100E70008A3C18F004C081E0089582E0089580E083
:100E80000895EF92FF920F931F93CF93DF938FE616
:100E900093E09F938F930E94DE0685E693E09F93F5
:100EA0008F930E94DE068AE593E09F938F930E94C2
:100EB000DE0604E611E00F900F900F900F900F9058
:100EC0000F90C0E0D0E089E4E82E83E0F82EF8012E
:100ED00080818823B1F091811F929F931F928F93FD
:100EE00082811F928F93DF93CF93FF92EF920E94A4
:100EF000DE06EDB7FEB73A960FB6F894FEBF0FBE0A
:100F0000EDBF21960D5F1F4FC031D10501F787E47A
:100F100093E09F938F930E94DE060F900F90DF91D6
:100F2000CF911F910F91FF90EF900895982F9F7789
:100F3000923081F038F4992351F0913089F480781F
:100F40008A640895933049F09F37B1F009C08078E2
:100F5000826408958078896408958078886408950B
:100F60001F928F9380EF92E09F938F930E94DE06F3
:100F70000F900F900F900F9080E008950F931F93A4
:100F8000CF93DF938FEA93E09F938F930E94DE06C7
:100F90000F900F90C1E0D0E002EA13E063E08C2FE5
:100FA0000E94DB0F009771F09F938F93DF93CF9395
:100FB0001F930F930E94DE060F900F900F900F90DB
:100FC0000F900F902196C031D10541F780EA93E050
:100FD0009F938F930E94DE060F900F90DF91CF9129
:100FE0001F910F910895FF920F931F93CF93DF935B
:100FF000F82E00910001109101018FEF9FEF909367
:101000000101809300010F3F8FEF180751F58F2DDD
:101010000E94FE0F8C01009709F472C01F938F93FA
:101020008F2D90E063E070E00E94002F8C599E4F5E
:10103000FC0181811F928F931F92FF9288E793E0BA
:101040009F938F930E94DE068DB79EB708960FB6CA
:10105000F8949EBF0FBE8DBF0F379FE7190769F445
:1010600008C00115110509F44BC00F37FFE71F0732
:1010700081F48FE70E94E70645C00F3FEFEF1E07A0
:1010800041F48FEF0E94E7060E94BE070E944107CD
:1010900039C0C12FD02F1F3F11F4C02FDFEF8F2D8C
:1010A00090E063E070E00E94002F8C599E4FFC019D
:1010B00081810E940707813061F48C2F8F77823302
:1010C00019F4C078CA6007C08A3029F4C078C263B6
:1010D00002C0823031F48C2F8F778A3211F4C078BD
:1010E000C0678C2F0E94E706DF3F61F08D2F90E0F4
:1010F000982F88278F6F909301018093000102C081
:1011000080E001C081E0DF91CF911F910F91FF90AE
:1011100008951F93CF93DF93182F0E94FE0FEC01C9
:10112000892B39F1DF93CF931F921F9381E093E0D6
:101130009F938F930E94DE068D2F99270F900F901B
:101140000F900F900F900F908F3F910529F00E9404
:10115000960781110E94E706CE0199278F3F9105DE
:1011600031F08C2F0E94960781110E94E70681E0E2
:1011700001C080E0DF91CF911F910895AF92BF929F
:10118000CF92DF92EF92FF920F931F93CF93DF9353
:1011900000D000D01F92CDB7DEB7D82E90E063E02C
:1011A00070E00E94002F8C599E4FFC01028125E0C7
:1011B000CE0101967C01AC0160E08D2D0E944A0FAA
:1011C000182F823008F4DBC11F920F931F92DF9219
:1011D00089E393E09F938F930E94DE060F900F9018
:1011E0000F900F900F900F906701F3E3AF2EF3E095
:1011F000BF2EF60181916F011F928F93BF92AF9224
:101200000E94DE068C2D8E190F900F900F900F907C
:10121000811778F380E393E09F938F930E94DE061B
:101220000F900F900C3449F5898191E0582F50743C
:1012300086FF90E02A81422F40743B8132FF02C03A
:101240008F7701C08068898330FF02C02F7701C08B
:1012500020682A8331FF02C088E001C088E88B83C0
:10126000552319F08B8180678B83442309F4D0C008
:101270008B8187608B8381E0CCC00D3481F49B81AE
:101280008A81292F87FF02C0206801C02F772B8316
:1012900097FF02C0806801C08F778A83A2C00234A2
:1012A00059F449813A811430D1F546FB992790F9D8
:1012B00036FB882780F9AAC00F3229F00F3519F0C4
:1012C000063609F05BC0498191E0642F607446FFE7
:1012D00090E03A8181E0532F507436FF80E02B81FB
:1012E00020FB47F94983422F42704295440F440F37
:1012F000407C3F77342B3A83322F34703295330F52
:10130000307E2870232B611102C030E001C030E72D
:10131000232B511102C030E05DC037E05BC091E08B
:10132000742F707446FF90E081E0632F607436FF85
:1013300080E02B81522F54705295550F507EE22F32
:10134000E295E07F5E234F77452B4983422F427021
:101350004295440F440F407C3F77342B3A8330E072
:101360003695322F222737952795711102C040E01C
:1013700001C040E7242B61112CC029C0033069F55E
:10138000498191E0642F607446FF90E03A8181E0EA
:10139000532F507436FF80E02B8120FB47F949839F
:1013A000422F44704295440F407E3F77342B3A835E
:1013B000227030E076E0220F331F7A95E1F7611159
:1013C00002C040E001C040E7242B511102C038E0C8
:1013D00001C03FE0232B2B831CC0043011F00233EB
:1013E00059F4FE01E10FF11D808186FB992790F9E8
:1013F00082FB882780F90EC0998196FB992790F986
:101400002A8126FB882780F920682A8312E002C0FF
:1014100080E013E048EF58E81530B1F0212F012E9D
:10142000000C330BF701E20FF31F911102C0508340
:1014300001C04083882331F0F701E20FF31F2081C0
:10144000276020831F5FE8CF2D8123FD02C080E845
:1014500001C080E027FF80644C8143FF806247FF2A
:1014600080616B8163FF886067FF84603A8137FF2A
:101470008260598157FF816080935F01A62FA0771A
:10148000B0E093E0AA0FBB1F9A95E1F7942F9077F5
:10149000E92FF0E076E0EE0FFF1F7A95E1F7EA2BF7
:1014A000FB2B5F77DF01A52BE22FE077F0E0FE2F2B
:1014B000EE27FF0FEA2BFB2B932F9F7730E0322F85
:1014C00022273295330F307E292B677070E0769596
:1014D000762F662777956795262B372B477050E038
:1014E000542F4427550F550F242B352B622F932F44
:1014F00021384FEF340714F461E89FEF462F592F3E
:101500004038510514F04FE750E0AE2F9F2FE138DF
:101510006FEFF60714F4A1E89FEF6A2F792F603878
:10152000710514F06FE770E010925B0110925C019E
:1015300010925D0110925E01109262014093600171
:10154000609361011F921F92FF93EF937F936F93BC
:101550003F932F935F934F931F928F938DE093E070
:101560009F938F930E94DE068FE591E00E941D19E4
:101570000FB6F894DEBF0FBECDBF81E001C080E0A2
:101580000F900F900F900F900F90DF91CF911F91C0
:101590000F91FF90EF90DF90CF90BF90AF900895A4
:1015A00080915F01089580919503816080939503F8
:1015B000E4E6F1E0108211821282339681E0E43990
:1015C000F807C1F7E4E9F1E084EA91E011928E179F
:1015D0009F07E1F7569A5E9A0E943A0F0E94721096
:1015E0000E94BE07569A5E980895089580E0089577
:1015F000E82FF0E0EC56FE4F80810895FF920F93A4
:101600001F93CF93DF93C82F04E611E0DFE0F82E9D
:10161000F094F80185A5823021F46F2D8D2F0E9462
:101620007B10D15003501109D73099F76C2F60957A
:1016300082E0DF91CF911F910F91FF900C947B106E
:101640002F923F924F925F926F927F928F929F92D2
:10165000AF92BF92CF92DF92EF92FF920F931F93C0
:10166000CF93DF93CDB7DEB764970FB6F894DEBFA4
:101670000FBECDBFD09002018091590190915A01C7
:101680000E94AF260B9718F5809156019091570153
:101690000E94AF26883E934008F476C30E949726A6
:1016A000909357018093560184E691E09A8B898B41
:1016B0009C8B8B8BCC24C394D12C10E040901D01CB
:1016C00050901E0160901F0170902001B4C00E94D4
:1016D000972690935A018093590100E07E0189E09A
:1016E000E80EF11C92E9A92E93E0B92E2CE8822E87
:1016F00023E0922E39E8632E33E0732E1D2D1F70E8
:1017000009F46DC0C12ED12CC60163E070E00E94C7
:10171000002F8C599E4FFC018081823051F018F4CB
:10172000882371F01EC0833031F08730D1F4812FCF
:1017300015C0812F0DC0812F0E94BE08082F4BC0FD
:10174000133049F0173049F0123009F048C082E0F8
:101750000E94F307F3CF83E0EFCF87E00E94890870
:10176000EDCF28E0A70160E0812F0E944A0F582E9C
:10177000882389F1C60163E070E00E94002F8C5934
:101780009E4FFC0182811F928F93DF92CF92BF9276
:10179000AF920E94DE060F900F900F900F900F9067
:1017A0000F9067018C2D8E19851570F4F6018191CB
:1017B0006F011F928F939F928F920E94DE060F906F
:1017C0000F900F900F90EECF7F926F920E94DE06E7
:1017D0000F900F9001E00E94470F882339F0DD241D
:1017E000D394D10E10910201D11288CF1F701093A3
:1017F00002018091580181110BC00E943F0F81119D
:1018000010C08FE70E94E70681E08093580109C06D
:101810000E943F0F882329F08FEF0E94E706109265
:101820005801002309F430CF0E9497269093570166
:1018300080935601A9C28C2C63E0882D0E94DB0F97
:101840005C01009791F4EB89FC898381882309F47A
:1018500050C0C60163E070E00E94002F8C599E4F7B
:10186000FC0110821182128243C03C2C2D2CBF92AD
:101870008F93DF92CF928AED92E09F938F930E9495
:10188000DE060F900F900F900F900F900F90E4E6F0
:10189000F1E00FE010E0F02EE02E912E85A58823D8
:1018A00059F001501109339707301105A1F72F9214
:1018B0003F9283EC92E014C04B2D407F402B2EEFE3
:1018C00063E0882D0E944A1063E0802F0E94DB0FA6
:1018D0009C01892B09F046C02F923F928FEA92E03B
:1018E0009F938F930E94DE060F900F900F900F90A2
:1018F00011E02FEFC21AD20A8B899C8903969C8B28
:101900008B8B98E0C916D10409F095CF00E063E015
:101910008C2D0E94DB0F892B89F4E989FA89808D4F
:10192000882361F0C60163E070E00E94002F8C59AB
:101930009E4FFC0110821182128201E089899A89EE
:1019400003969A8B898B9FEFC91AD90AE0E1CE16CC
:10195000D104E9F6111103C0002309F415C20E9455
:10196000410712C2C80163E070E00E94002F8C5949
:101970009E4FFC018082C80163E070E00E94002F4E
:101980008C599E4FFC012183C80163E070E00E94E6
:10199000002F8C599E4FFC0122833F932F931F935E
:1019A0000F932F923F9283E992E09F938F930E942F
:1019B000DE060FB6F894DEBF0FBECDBF92E08912EF
:1019C0005DC063E0802F0E94DB0F5C01009729F46B
:1019D0001F930F9382E892E05FC0BF928F931F9393
:1019E0000F938CE692E09F938F930E94DE068A2DE0
:1019F0000E9407070F900F900F900F900F900F907D
:101A0000882339F0813041F0823049F482E391E05B
:101A100008C089E291E005C08EE291E002C086E351
:101A200091E09F938F939F92EF928AE592E09F932C
:101A30008F930E94DE0623E04B2D63E08F2D0E94E2
:101A40004A1063E08F2D0E94DB0F282F8E2D992DD9
:101A500063E070E00E94002F8C599E4FFC012283AE
:101A60000E94C818682F60958F2D0E947B100F90E0
:101A70000F900F900F900F900F9084C1F3E08F1292
:101A800070C163E0802F0E94DB0F5C01009769F456
:101A90001F930F9389E492E09F938F930E94DE0639
:101AA0000F900F900F900F906DC1BF928F931F9367
:101AB0000F9383E392E09F938F930E94DE061A2D8B
:101AC0000F900F900F900F900F900F901F3231F0EA
:101AD0001F3521F0163611F0123461F449825A8212
:101AE0006B827C8224E0AE014F5F5F4F61E08F2DFF
:101AF0000E9401108FEF810F823008F040C024E077
:101B00004B2D63E08F2D0E944A1063E08F2D0E94C1
:101B1000DB0F5C01182F8430A9F123E04B2D63E02B
:101B20008F2D0E944A1063E08F2D0E94DB0F5C0115
:101B3000182F833039F427E040E062E08F2D0E94B7
:101B40004A1004C1813099F422E04B2D63E08F2DBF
:101B50000E944A1063E08F2D0E94DB0F5C01182F5A
:101B6000813029F49F92EF928CE192E006C012300E
:101B700031F49F92EF9285E092E09F93C1C01430C0
:101B800009F0C2C028E0AE014F5F5F4F61E08F2DCA
:101B90000E944A0F863030F02D813E813227232764
:101BA000322704C0882369F124E630E098851F922B
:101BB0008F931F929F933F932F931F929F938F8199
:101BC0001F928F938E811F928F938D811F928F937F
:101BD0008C811F928F938B811F928F938A811F928A
:101BE0008F9389811F928F939F92EF928AEB91E05E
:101BF0009F938F930E94DE060FB6F894DEBF0FBE50
:101C0000CDBF89818B34C1F58A818D3479F48B8184
:101C10008C3409F070C08C81813309F06CC09F92C4
:101C2000EF92E4EAF1E0FF93EF936BC08F3409F099
:101C300062C08B81893409F05EC08C81843509F0E3
:101C40005AC08F2D0E945C1022E44B2D63E08F2D33
:101C50000E944A1063E08F2D0E94DB0F182F9F9285
:101C6000EF9280E991E09F938F930E94DE060F90A0
:101C70000F900F900F9048C08A3951F58A81805299
:101C80008230C8F59F92EF9280E891E09F938F9306
:101C90000E94DE0621E840E061E08F2D0E944A109C
:101CA00021E841E061E08F2D0E944A1021E842E0E6
:101CB00061E08F2D0E944A1028E343E061E08F2D00
:101CC0000E944A100F900F900F900F901CE43EC09E
:101CD0008C3489F48A81843571F49F92EF9287E67F
:101CE00091E09F938F930E94DE060F900F900F90CC
:101CF0000F901DE42BC09F92EF9287E591E09F9398
:101D00008F930E94DE061EC0123301F59F92EF9260
:101D100085E491E09F938F930E94DE0688E0E1E2E4
:101D2000F1E0DE01119601900D928A95E1F78F2D79
:101D30000E945C1028E0AE014F5F5F4F62E08F2D84
:101D40000E9401100F900F900F900F908E2D992DE3
:101D500063E070E00E94002F8C599E4FFC011283BB
:101D600011C0F7E08F120EC01F930F9388E291E02D
:101D70009F938F930E94DE0611E00F900F900F90BB
:101D80000F905ACD11E058CD64960FB6F894DEBF8F
:101D90000FBECDBFDF91CF911F910F91FF90EF90BC
:101DA000DF90CF90BF90AF909F908F907F906F907B
:101DB0005F904F903F902F900895509A83E091E06C
:101DC0000197F1F700C0000050989AEB9A95F1F74F
:101DD00000C00895509A8AEB8A95F1F700C0509898
:101DE00083E091E00197F1F700C000000895EF92C1
:101DF000FF920F931F93CF93DF93C0E0D0E090E862
:101E0000E92EF12C082F10E0C7010C2E02C0959589
:101E100087950A94E2F780239123892B19F00E9479
:101E2000EA0E02C00E94DD0E2196C830D10561F78E
:101E3000DF91CF911F910F91FF90EF900895509AED
:101E400083EF9BE00197F1F700C000000C94EA0ECD
:101E5000489B06C023E02A95F1F700000197C1F7DF
:101E60000895489906C023E02A95F1F700000197EC
:101E7000C1F7089558985098599A51980895599AC9
:101E8000519889B18695817008950895089580913B
:101E9000A4010895EF92FF920F931F93CF93DF93C6
:101EA000182FC62F7A01D22F80E0422F50E0282F22
:101EB000082E000C330B2417350734F4F701E20F1A
:101EC000F31F10828F5FF3CFF8940E941F0F812FB2
:101ED0008295807FCC608C2B0E94F70E0E94DD0ED5
:101EE000489904C081E08093A40102C01092A4012B
:101EF00084EF91E00E94310F892B19F48BEB93E072
:101F00001AC084EF91E00E94280F892B19F478946D
:101F100080E04AC088E290E00E94310F892B19F4DA
:101F200089EB93E008C084E690E00E94280F892B9B
:101F300051F487EB93E09F938F930E94DE06789491
:101F40000F900F90E5CFC0E082E890E00E94310F43
:101F50008823F9F08C011127C8010E94280F8823DB
:101F6000C1F09C2F9695969596959D1780F4F70154
:101F7000E90FF11D9081990F22E830E0201B310B11
:101F8000081B1109201731070CF491609083CF5F73
:101F9000D9F678948FE193E00197F1F700C0000043
:101FA0008C2F869586958695DF91CF911F910F9105
:101FB000FF90EF900895CF93DF93CDB7DEB72897CA
:101FC0000FB6F894DEBF0FBECDBF28E0AE014F5F65
:101FD0005F4F0E944A0F823031F489819A8198279D
:101FE0008927982702C080E090E028960FB6F894E1
:101FF000DEBF0FBECDBFDF91CF91089560E00C949E
:10200000DB0FEF92FF921F93CF93DF93182FD62F02
:102010007A01C22FF8940E941F0F812F8295807F32
:10202000D8608D2B0E94F70E0E94DD0E489904C0E7
:1020300081E08093A40102C01092A40184EF91E09A
:102040000E94310F8FE193E00197F1F700C000008B
:102050000E94EA0E10E0D0E0812F012E000C990BB7
:102060008C179D0744F4F701E80FF91F80810E9447
:10207000F70E1F5FF1CF0E94DD0E78948FE193E0A1
:102080000197F1F700C00000DF91CF911F91FF9001
:10209000EF900895CF93DF9300D0CDB7DEB749839B
:1020A0002A8322E0AE014F5F5F4F0E9401100F9024
:1020B0000F90DF91CF910895CF93C82FF8940E948D
:1020C0001F0F8C2F8295807F81600E94F70E0E94E7
:1020D000DD0E8FE193E00197F1F700C000007894E6
:1020E000CF910895509A8FED9EE20197F1F700C0CD
:1020F000000050980895CF93DF93D82FC62F62E049
:102100000E94DB0FEFE3F6E03197F1F700C000002B
:10211000282F287FC7702C2B492F62E08D2FDF914D
:10212000CF910C944A108091B1020895CF93DF9320
:1021300000D01F92CDB7DEB72091AA03243021F53D
:1021400023E029839B838A8382E08093E9008FEFD9
:102150009091E800815095FD06C095ED9A95F1F7B4
:1021600000008111F5CF8091E80085FF0DC040E0AF
:1021700050E063E070E0CE0101960E94341580913A
:10218000E8008E778093E8000F900F900F90DF911A
:10219000CF910895CF93DF9300D01F92CDB7DEB7D4
:1021A0002091AA03243061F519821A821B8222E051
:1021B00029838138910520F0805891099B838A8377
:1021C00082E08093E9008FEF9091E800815095FDC7
:1021D00006C095ED9A95F1F700008111F5CF809139
:1021E000E80085FF0DC040E050E063E070E0CE0104
:1021F00001960E9434158091E8008E778093E80064
:102200000F900F900F90DF91CF9108952091AA0326
:10221000243051F522E02093E9002FEF3091E800BF
:10222000215035FD06C035ED3A95F1F7000021113A
:10223000F5CF2091E80025FF17C02091130122233C
:1022400041F021E02093F10040E050E065E070E0D3
:1022500004C040E050E063E070E00E9434158091DB
:10226000E8008E778093E8000895CF93DF93209164
:10227000AA03243049F521E02093E90021E8215008
:1022800059F03091E80035FD07C0EFE3F1E03197F8
:10229000F1F700C00000F3CF2091E80025FF14C043
:1022A000EC0140E050E068E070E00E94341580915D
:1022B000E8008E778093E80088E0FE01A9EAB2E0AA
:1022C00001900D928A95E1F7DF91CF910895CF9318
:1022D000C091A701C1110BC00E94A326643C7940A4
:1022E0008105910520F081E08093A701C1E08C2F4A
:1022F000CF910895FF920F931F93CF93DF93D82F21
:102300000FB607FE83C08091AA03843081F08091CC
:10231000060190E001962091080130E0822393238A
:102320002091070130E08217930709F0C9C00E948D
:102330006711811110C08091060190E001962091F3
:10234000080130E0822393232091070130E08217B7
:10235000930709F0B5C00E9497268C01C091E9004F
:10236000CF709091EC00892F817090FD80E8C82B90
:1023700083E08093E90085E0F82E8091EB0085FDF5
:1023800042C08091EB0080FF3EC08091EE0087FF4D
:102390003AC08091070190910601981709F457C03F
:1023A0009091E80095FF8AC0E0910401F091050149
:1023B000E80FF11D20818F5F9091080189238093A0
:1023C00007012093F1008091E80085FDE2CF809124
:1023D000E80080FFDECF8091E8008E778093E800F0
:1023E000F0920301D6CF8091060190E001962091F2
:1023F000080130E0822393232091070130E0821707
:10240000930709F448C0CF70C093E90040910601DA
:10241000842F90E001962091080130E082239323DD
:102420002091070130E08217930709F44CC0E09136
:102430000401F0910501E40FF11DD08380910601A4
:102440008F5F909108018923809306013CC08091A1
:10245000E80085FF33C0D093F10081E09091F20055
:10246000992391F09091E80090FF0EC09091E800C0
:1024700095FF03C01092F100F9CF9091E8009E778C
:102480009093E800F0920301882309F4ACCFCF7059
:10249000C093E90018C080910301882309F4B3CFE9
:1024A0000E9497269C018017910711F4890165CF3E
:1024B00090910301915090930301F8CF80E0CECF2B
:1024C00040910601B4CF80E0DF91CF911F910F9131
:1024D000FF900895089542E061EC81E00E94AD1400
:1024E00042E061EC82E00E94AD1446E261EC83E0E0
:1024F0000C94AD148091AC03833009F453C030F4D4
:10250000813071F0823009F4BAC008958A3009F43C
:10251000A6C08B3009F478C0893009F0C8C020C04B
:102520008091AB03813A09F0C2C08091E800877FB7
:102530008093E8008091AF039091B003892B21F440
:1025400068E089EA92E003C060E080E090E070E03B
:102550000E9481158091E8008B778093E8000895B0
:102560008091AB03813209F0A2C08091AF039091BA
:10257000B003892B09F09BC08091E800877F80938E
:10258000E8008091E80082FD05C08091AA038111D6
:10259000F8CF8DC08091F1008093B1028091E80066
:1025A0008B7781C08091AB03813A09F080C0809124
:1025B000AF039091B003892BA1F48091E800877F4D
:1025C0008093E8008091E80080FFFCCF80911401A7
:1025D0008093F1008091E8008E778093E8000E945C
:1025E000E2148091AF039091B003019709F05FC0AE
:1025F0008091E800877F8093E8008091E80080FF69
:10260000FCCF809113014AC08091AB03813209F065
:102610004EC08091AF039091B003892B69F48091F3
:10262000E800877F8093E8000E94E2148091AD0368
:10263000809314010E94481C8091AF039091B003D5
:102640000197A9F58091E800877F8093E8000E94B8
:10265000E2148091AD03809313010C94481C809187
:10266000AB03813221F58091E800877F8093E800F9
:102670000E94E2148091AE038093B202089580918B
:10268000AB03813AA1F48091E800877F8093E80052
:102690008091E80080FFFCCF8091B2028093F1002E
:1026A0008091E8008E778093E8000C94E2140895FE
:1026B0008091B1028093A8011092B1020E94491A40
:1026C0000C94481C0C9458130E9424268091A80353
:1026D000882329F00E944D2681110C9497140895A7
:1026E0000E9461268091A8018093B10208950C9404
:1026F000701308950C947913CF9384B7877F84BFA8
:102700000FB6F894A895809160008861809360006E
:10271000109260000FBE90E080E80FB6F8948093AE
:102720006100909361000FBE8AE791E10E94F72556
:1027300089E091E00E94C3188DED93E00E94450668
:102740000E947A130E949A190E949A170E94ED170C
:1027500078940E949C198091AA03843029F00E94E9
:10276000A8180E947913F7CF0E9467118823B9F344
:102770008BEC93E00E9445060E94D30A8DEB93E018
:102780000E944506C3E08091AA03853019F40E9497
:102790006413F9CF0E94200B0E94A2192091E4003B
:1027A0003091E5008091A5019091A6012817390785
:1027B00009F464C08091E4009091E5009093A60133
:1027C0008093A5010E946711882309F457C0809166
:1027D000AA03843009F052C08091E9008F702091E3
:1027E000EC00922F917020FD90E8892BC093E900B6
:1027F0009091EB0090FF3FC09091EE0097FF3BC09F
:102800009091070120910601291709F12091E80014
:1028100025FF1DC0E0910401F0910501E90FF11DB4
:1028200030819F5F2091080192239093070130939C
:10283000F1009091E80095FDE3CF9091E80090FFC2
:10284000DFCF9091E8009E779093E800D9CF9091E8
:10285000F200992381F09091E80090FF0CC09091D4
:10286000E80095FF03C01092F100F9CF9091E800C5
:102870009E779093E8008F708093E9000E94A818DB
:1028800082CF292F332723303105C9F060F421305E
:10289000310581F02230310509F041C084E590E036
:1028A0002AE334E040C021323105E1F02232310523
:1028B00031F135C082E190E02EE834E034C0992750
:1028C0008130910549F028F0029749F5E6EFF3E0F1
:1028D00005C0E6E3F4E002C0E6E2F4E0849190E0B3
:1028E0009F0121C063307105D0F4660F771FFB0193
:1028F000ED5BFE4F2081318189E090E014C06330B0
:10290000710568F4FB01EE0FFF1FE35CFE4F2081B1
:102910003181FB01E65CFE4F808190E004C080E0E5
:1029200090E020E030E0FA0131832083089584E0D4
:1029300089BD86E089BD09B400FEFDCF8091D80035
:102940008F7D8093D8008091E00082608093E000CA
:102950008091E00081FDFCCF0895982F953068F5B7
:102960009093E900981739F07091EC002091ED00F8
:102970005091F00003C0242F762F50E021FD02C0BB
:102980009F5FECCF3091EB003E7F3093EB003091B6
:10299000ED003D7F3093ED003091EB0031603093DE
:1029A000EB007093EC002093ED005093F000209129
:1029B000EE0027FDE5CF80E008958F708093E90059
:1029C00081E008958091AB0387FF11C08091E800FA
:1029D00082FD05C08091AA038111F8CF11C08091BA
:1029E000E8008B770BC08091AA03882349F080917F
:1029F000E80080FFF8CF8091E8008E778093E800B0
:102A000008952091E4003091E50095E64091EC00B6
:102A1000842F817040FF23C08091E80080FD1DC09D
:102A20008091AA03882399F0853099F08091EB007A
:102A300085FD11C04091E4005091E5002417350751
:102A400029F3915011F09A01E1CF84E0089582E0DA
:102A5000089583E0089581E0089580E0089540910D
:102A6000E80042FFDDCF0895CF92DF92EF92FF9210
:102A70000F931F93CF93DF93EC018B017A010E9498
:102A80000115811135C0E114F10439F0F70180819D
:102A90009181081B190BC80FD91FC12CD12C01150E
:102AA000110529F18091E80085FD18C08091E800AA
:102AB0008E778093E8000E94A818E114F10449F091
:102AC000F70180819181C80ED91ED182C08285E034
:102AD0000FC00E940115882311F30AC089918093C9
:102AE000F10001501109FFEFCF1ADF0AD8CF80E0C3
:102AF000DF91CF911F910F91FF90EF90DF90CF90DA
:102B000008952091B1033091B2032617370748F09A
:102B10006115710539F42091E8002E772093E800C3
:102B200001C0B901FC0120E06115710561F18091DE
:102B3000AA038823D9F18530D9F18091E80083FD7B
:102B400039C08091E80082FD2BC08091E80080FFB1
:102B5000EBCF8091F20090E06115710551F0883063
:102B6000910538F421912093F1006150710901968B
:102B7000F3CF21E0089709F020E08091E8008E77FC
:102B80008093E800D1CF2111D2CF0AC08091AA034F
:102B9000882361F0853061F08091E80083FD0AC0F0
:102BA0008091E80082FFF2CF80E0089582E00895EE
:102BB00083E0089581E008952091B1033091B2033C
:102BC0002617370748F06115710539F42091E800A0
:102BD0002E772093E80001C0B901FC0120E06115C7
:102BE000710579F18091AA03882309F43DC08530ED
:102BF00009F43CC08091E80083FD3AC08091E80070
:102C000082FD2CC08091E80080FFE9CF8091F20026
:102C100090E06115710559F08830910540F42491D8
:102C20002093F1003196615071090196F2CF21E0B5
:102C3000089709F020E08091E8008E778093E80003
:102C4000CECF2111CFCF0AC08091AA03882361F093
:102C5000853061F08091E80083FD0AC08091E80032
:102C600082FFF2CF80E0089582E0089583E0089526
:102C700081E008951F93CF93DF93CDB7DEB7AA9776
:102C80000FB6F894DEBF0FBECDBFEBEAF3E0809144
:102C9000F100819323E0E33BF207C9F70E947A1227
:102CA0008091E80083FF2EC18091AB039091AC032B
:102CB000492F50E04A30510508F024C1FA01E65C82
:102CC000FF4F0C94252F803821F0823809F01AC16B
:102CD00008C08091A7039091A803992389F082608E
:102CE0000FC08091AF038F70853008F00BC18093C7
:102CF000E9008091EB0085FB882780F91092E900BC
:102D00009091E800977F9093E8008093F1001092F3
:102D1000F100D1C0282F2D7F09F0F4C0882319F0CD
:102D2000823061F0EFC08091AD03813009F0EAC0DC
:102D3000933009F080E08093A8032EC08091AD030A
:102D400081112AC08091AF038F702FEF280F24309C
:102D500008F0D8C08093E9002091EB0020FF1CC050
:102D6000933021F48091EB00806214C09091EB00CD
:102D700090619093EB0021E030E0A90102C0440F84
:102D8000551F8A95E2F74093EA001092EA0080917D
:102D9000EB0088608093EB001092E9008091E800DE
:102DA000877F8093E8000E94E214ACC08111AAC022
:102DB0001091AD031F778091E3008078812B809381
:102DC000E3008091E800877F8093E8000E94E2148E
:102DD0008091E80080FFFCCF8091E30080688093C1
:102DE000E300111102C082E001C083E08093AA03D6
:102DF00089C08058823008F085C08091AD039091E1
:102E0000AE038C3D53E0950779F583E08A838AE22F
:102E100089834FB7F894DE01139620E03EE051E23B
:102E2000E32FF0E050935700E49120FF03C0E295B8
:102E3000EF703F5FEF708E2F90E0EA3010F0C79692
:102E400001C0C0968D939D932F5F243149F74FBFEA
:102E50008091E800877F8093E8006AE270E0CE010D
:102E600001960E94811516C06091AF037091B00366
:102E7000AE014F5F5F4F0E944114BC01892B09F4E2
:102E800041C09091E800977F9093E80089819A81F2
:102E90000E94DC158091E8008B778093E80032C0B7
:102EA000803881F58091E800877F8093E8008091E9
:102EB000A6038093F1008091E8008E7772CF811194
:102EC00021C08091AD039091AE0399270297D4F46D
:102ED0008091E800877F8093E8008091AD03809324
:102EE000A6030E94E2148091A603811106C080917E
:102EF000E30087FD02C081E001C084E08093AA0363
:102F00000E946B128091E80083FF0AC08091E80064
:102F1000877F8093E8008091EB0080628093EB00D4
:102F2000AA960FB6F894DEBF0FBECDBFDF91CF914A
:102F30001F9108950E94F7170E94FA17E0EEF0E043
:102F4000808181608083E8EDF0E080818F778083ED
:102F500019BCE3E6F0E08081816080831092A903D0
:102F600008950E94F7170E94FA178091D8008F7772
:102F70008093D8008091D80080688093D800809199
:102F8000D8008F7D8093D80084E089BD86E089BD1C
:102F900009B400FEFDCF1092AA031092A60310926E
:102FA000A8031092A70342E060E080E00E94AD1405
:102FB0008091E1008E7F8093E1008091E20081604A
:102FC0008093E2008091E20088608093E20080912B
:102FD000E0008E7F8093E0000895E3E6F0E08081DA
:102FE0008E7F808381E08093A9030C94B1171092A7
:102FF000E20008951092E10008951F920F920FB61B
:103000000F9211242F933F934F935F936F937F936E
:103010008F939F93AF93BF93EF93FF938091E100C2
:1030200082FF0BC08091E20082FF07C08091E10027
:103030008B7F8093E1000E94A7188091E10080FFC0
:1030400019C08091E20080FF15C08091E2008E7F60
:103050008093E2008091E20080618093E2008091A1
:10306000D80080628093D80019BC85E08093AA03C1
:103070000E9462138091E10084FF30C08091E200E1
:1030800084FF2CC084E089BD86E089BD09B400FEC0
:10309000FDCF8091D8008F7D8093D8008091E10092
:1030A0008F7E8093E1008091E2008F7E8093E2002A
:1030B0008091E20081608093E2008091A6038823E2
:1030C00011F084E007C08091E30087FD02C081E039
:1030D00001C083E08093AA030E9477138091E100EE
:1030E00083FF24C08091E20083FF20C08091E10033
:1030F000877F8093E10082E08093AA031092A60369
:103100008091E1008E7F8093E1008091E2008E7FCC
:103110008093E2008091E20080618093E20042E0CF
:1031200060E080E00E94AD140E946A12FF91EF916E
:10313000BF91AF919F918F917F916F915F914F91CF
:103140003F912F910F900FBE0F901F9018950895EB
:10315000CF938091AA038823A1F0C091E900CF709A
:103160009091EC00892F817090FD80E8C82B10921F
:10317000E9008091E80083FD0E943A16CF70C09369
:10318000E900CF9108959093B8028093B702089513
:10319000E091B702F091B802309721F00190F081F0
:1031A000E02D099480E00895EF92FF920F931F9312
:1031B000CF93DF93E091B702F091B8023097B1F16D
:1031C0008C010280F381E02D09958091950382FFA7
:1031D0002DC080FF04C087EA95E00E944506E80103
:1031E00018E081EAE82E85E0F82E8091950380FFB3
:1031F0000BC088811F928F93FF92EF920E94DE0690
:103200000F900F900F900F90115021961111EDCF4C
:103210008091950380FF0AC08FE995E0DF91CF91FF
:103220001F910F91FF90EF900C944506DF91CF9185
:103230001F910F91FF90EF9008951F93CF93DF930D
:103240002091B7023091B802232BB1F0EC01188124
:103250000E94F8299881892B88830E94D00A98813E
:10326000892B8883E091B702F091B8020480F58140
:10327000E02DCE0109951883DF91CF911F9108951C
:10328000CF93DF932091B5023091B602281739070A
:1032900009F19093B6028093B502E091B702F091E4
:1032A000B8023097B9F0EC010680F781E02D09955E
:1032B0008091950382FF0EC080FF0CC0DF93CF93F7
:1032C00081E995E09F938F930E94DE060F900F9007
:1032D0000F900F90DF91CF910895CF93DF932091BE
:1032E000B3023091B4022817390709F19093B40260
:1032F0008093B302E091B702F091B8023097B9F031
:10330000EC010084F185E02D09958091950382FF01
:103310000EC080FF0CC0DF93CF9381E895E09F93B0
:103320008F930E94DE060F900F900F900F90DF9109
:10333000CF9108950C944A1A0E948E260E94F50A95
:103340000C94450FBF92CF92DF92EF92FF920F93B2
:103350001F93CF93DF9300D000D01F92CDB7DEB77D
:103360000E94F60A0AEB12E0F12C8F2D0E94F80A57
:10337000B82EF801C080C82639F4F3940F5F1F4FB0
:10338000F0E1FF12F2CF30C08091950381FD0E94E1
:103390005F1AD12CEE24E3948C2D8E21F9F0D98282
:1033A000FA8291E08B2D8E2109F490E09B830E949C
:1033B00097268160782F9D838C8349815A816B8108
:1033C0008D810E94951A49815A816B817C818D8102
:1033D0000E940F26F80180818E258083D394EE0C05
:1033E000F8E0DF12D9CFC9CF8FEF89838A831B82A0
:1033F0000E9497268160782F9D838C8349815A8112
:103400006B818D810E94951A0E940E260E9446298A
:103410000E94460F0E94C8189091B902891741F185
:103420000E94C8188093B9029091950392FF0EC034
:1034300090FF0CC01F928F9382EB95E09F938F9328
:103440000E94DE060F900F900F900F908091B902AE
:103450000F900F900F900F900F90DF91CF911F91D1
:103460000F91FF90EF90DF90CF90BF900C942026AB
:103470000F900F900F900F900F90DF91CF911F91B1
:103480000F91FF90EF90DF90CF90BF9008950C9434
:10349000FE0A08950895CF93C62F0E94F80A21E0EE
:1034A00030E002C0220F331FCA95E2F790E02823D4
:1034B000392381E0232B09F480E0CF910895EF9226
:1034C000FF920F931F93CF93DF9388EC95E00E94B8
:1034D0004506C0E0D0E089E3E82E81E0F82E0DEB50
:1034E00015E08C2F0E94F80A0E94FC25FF92EF92B3
:1034F0001F928F93DF93CF931F930F930E94DE064B
:1035000021968DB79EB708960FB6F8949EBF0FBE52
:103510008DBFC031D10529F7DF91CF911F910F9158
:10352000FF90EF90089508950895CF93DF93CDB75E
:10353000DEB72B970FB6F894DEBF0FBECDBF942F2A
:103540004F83252F588769877A878B874A855B85C4
:10355000452B31F02F3F31F481E09F3F19F403C038
:1035600081E001C080E080FD07C04F8158856985FA
:103570007A858B850E940F26DE01119686E0FD017B
:1035800011928A95E9F785E0FE01379601900D9238
:103590008A95E1F749815A816B817C818D819E8179
:1035A0000E9465222B960FB6F894DEBF0FBECDBFEA
:1035B000DF91CF910895CF93DF93882309F4EEC074
:1035C000C82F8EE78C0F833018F5C23829F0C33826
:1035D00031F0C4E0D7E405C0C2E0D9E302C0C1E0E5
:1035E000D3E50E94C8188C2309F0D8C08D2F0E9403
:1035F00059250E94D1252FEF81EE94E02150804083
:103600009040E1F700C000008D2F0E9476250CC08D
:103610008CEF8C0F813A60F48C2F0E94742C8111F6
:10362000BDC08C2F0E945925DF91CF910C94D125DC
:1036300080E28C0F883048F4C77081E001C0880FA9
:10364000CA95EAF70E949725EFCF8BE58C0F833060
:1036500080F4C53A29F0C63A31F083E890E005C01D
:1036600081E890E002C082E890E0DF91CF910C9475
:10367000401988E58C0F873108F090C0C83A09F4EA
:1036800045C0C93A09F445C0CA3A09F445C0CB3A25
:1036900009F445C0CC3A09F445C0CD3A09F445C017
:1036A000CE3A09F445C0CF3A09F445C0C13B09F40C
:1036B00045C0C03B09F445C0C23B09F445C0C33B0B
:1036C00009F445C0C43B09F445C0C53B09F445C0F5
:1036D000C63B09F445C0C73B09F445C0C83B09F4E3
:1036E00045C0C93B09F445C0CA3B09F445C0CB3BC2
:1036F00009F445C0CC3B09F445C0CD3B09F445C0B5
:10370000CE3B09F445C080E090E044C082EE90E0FA
:1037100041C089EE90E03EC08AEE90E03BC085EB70
:1037200090E038C086EB90E035C083EB90E032C08B
:1037300084EB90E02FC087EB90E02CC08CEC90E005
:1037400029C08DEC90E026C083E891E023C08AE890
:1037500091E020C082E991E01DC084E991E01AC0A7
:1037600081E292E017C083E292E014C084E292E02A
:1037700011C085E292E00EC086E292E00BC087E2C3
:1037800092E008C08AE292E005C08FE690E002C0B5
:1037900080E790E0DF91CF910C946D19DF91CF918C
:1037A0000895CF93DF93882309F44FC09EE7980FC5
:1037B000933000F5823829F0833831F0C4E0D7E443
:1037C00005C0C2E0D9E302C0C1E0D3E50E94C81839
:1037D0008C23D9F18D2F0E9459250E94D1252FEFDE
:1037E00081EE94E0215080409040E1F700C000005D
:1037F0008D2F04C09CEF980F913A18F40E94762503
:103800000DC090E2980F983068F4877091E001C085
:10381000990F8A95EAF7892F0E949D25DF91CF9114
:103820000C94D1259BE5980F933030F480E090E024
:10383000DF91CF910C944019885A873130F480E0A1
:1038400090E0DF91CF910C946D19DF91CF910895A5
:10385000882321F00E9497250C94D1250895882370
:1038600021F00E949D250C94D12508950E94B72532
:103870000E9486250E94D1250E94EC290E94B92829
:1038800080E090E00E94401980E090E00C946D1977
:103890000E94A7250C94361CCF92DF92EF92FF92E4
:1038A0000F931F93CF93DF9300D000D01F92CDB71B
:1038B000DEB76C010E942226811118C385E0F60153
:1038C000DE01119601900D928A95E1F7F601408193
:1038D0005181238134812115310531F05F3F31F46D
:1038E00081E04F3F19F403C081E001C080E080FD1A
:1038F000FDC2F601F280E580E2948FE0E822498380
:103900005A83FB82722F3D832C836F2D8D810E9401
:10391000CE248C010E94CD240E94BD23E12FE2958C
:10392000EF708E2F90E0FC01EC5BFF4F0C94252F85
:10393000812F807F1F70882311F01295107FFF2048
:10394000B9F0112329F0812F0E94AA250E94D125C8
:10395000802F0F900F900F900F900F90DF91CF91CD
:103960001F910F91FF90EF90DF90CF900C94DB1A96
:10397000802F0E94D11B112309F4B8C2812F0E940D
:10398000B0250F900F900F900F900F90DF91CF9177
:103990001F910F91FF90EF90DF90CF900C94D12565
:1039A000812F807F1F70803211F01295107F0023CD
:1039B00019F0013009F12BC0FF20A9F0EE2059F1D8
:1039C000F1E0812FEF1228C00F900F900F900F9011
:1039D0000F90DF91CF911F910F91FF90EF90DF90AB
:1039E000CF900C94BA25EE2021F021E0E21609F4E4
:1039F0007DC20E94BD254DC0FF20E9F085E08E15F7
:103A000008F474C20E949425812329F042C0FF204B
:103A1000F1F1E11015C0812F0F900F900F900F90D2
:103A20000F90DF91CF911F910F91FF90EF90DF905A
:103A3000CF900C94281C94E09E1508F457C229C01E
:103A4000F601858180FF13C08F708583E4CF003F2E
:103A500009F489C108F055C180E4800F803208F470
:103A600059C1FF2009F4EAC1EE2009F49AC1802F60
:103A70000E94DB1A093309F0DAC1FFEF21EE84E07E
:103A8000F15020408040E1F700C000002FC2E1105B
:103A9000D7C1812F59C1812F86958695837019F0E2
:103AA0008130B9F023C2FF2019F0C801937002C021
:103AB00080E090E00F900F900F900F900F90DF91AB
:103AC000CF911F910F91FF90EF90DF90CF900C94CA
:103AD0004019FF2019F0C801937002C080E090E007
:103AE0000F900F900F900F900F90DF91CF911F913B
:103AF0000F91FF90EF90DF90CF900C946D19802F75
:103B0000FF2019F00E94CC2702C00E9434280F9099
:103B10000F900F900F900F90DF91CF911F910F9109
:103B2000FF90EF90DF90CF900C94B928812F837095
:103B300009F070C0F110DAC1202F22952695277068
:103B4000220F220F602F6F70862F90E0A0E0B0E070
:103B50006C017D01022E04C0CC0CDD1CEE1CFF1C90
:103B60000A94D2F704FF12C08FE090E0A0E0B0E02A
:103B700004C0880F991FAA1FBB1F2A95D2F7BC014A
:103B8000CD01609570958095909503C060E070E0E0
:103B9000CB011695169513701230B1F040F56C29D3
:103BA0007D298E299F29113031F10F900F900F90B0
:103BB0000F900F90DF91CF911F910F91FF90EF9099
:103BC000DF90CF900C94E2236C297D298E299F29C8
:103BD0000F900F900F900F900F90DF91CF911F914A
:103BE0000F91FF90EF90DF90CF900C94FC230E94F8
:103BF000E223C701B6010F900F900F900F900F9026
:103C0000DF91CF911F910F91FF90EF90DF90CF90B8
:103C10000C94C823FF2019F0812F817001C0869574
:103C2000882309F463C1202F229526952770220F3F
:103C3000220F602F6F70862F90E0A0E0B0E06C0143
:103C40007D01022E04C0CC0CDD1CEE1CFF1C0A946E
:103C5000D2F704FF12C08FE090E0A0E0B0E004C013
:103C6000880F991FAA1FBB1F2A95D2F7BC01CD014F
:103C7000609570958095909503C060E070E0CB01F1
:103C80001695169513701230B1F040F56C297D2908
:103C90008E299F29113031F10F900F900F900F90C6
:103CA0000F90DF91CF911F910F91FF90EF90DF90D8
:103CB000CF900C94A9246C297D298E299F290F90DF
:103CC0000F900F900F900F90DF91CF911F910F9158
:103CD000FF90EF90DF90CF900C94BB240E94A9241A
:103CE000C701B6010F900F900F900F900F90DF91CA
:103CF000CF911F910F91FF90EF90DF90CF900C9498
:103D00009724023F09F45EC008F449C0033F09F458
:103D10006CC0A7CE902F9071E92E812F8F71FF205C
:103D200051F00E943024802FEE2019F08295807F80
:103D300073CE8F7071CE0E945124802FEE2019F027
:103D40008295807F01C08F700F900F900F900F9021
:103D50000F90DF91CF911F910F91FF90EF90DF9027
:103D6000CF900C942F1CFF20A9F0E4E0EE1508F48E
:103D7000BDC0812F8F710F900F900F900F900F90FB
:103D8000DF91CF911F910F91FF90EF90DF90CF9037
:103D90000C947624F5E0FE1508F4A8C0EACFFF20C5
:103DA00099F0812F8F710F900F900F900F900F90BF
:103DB000DF91CF911F910F91FF90EF90DF90CF9007
:103DC0000C943024FF2069F3812F8F710F900F9096
:103DD0000F900F900F90DF91CF911F910F91FF9057
:103DE000EF90DF90CF900C945124FF2089F0812F29
:103DF0008F710F900F900F900F900F90DF91CF91D8
:103E00001F910F91FF90EF90DF90CF900C941B24A7
:103E10000F900F900F900F900F90DF91CF911F9107
:103E20000F91FF90EF90DF90CF900C941624033504
:103E300009F423CE073409F059C01FCEEE2021F239
:103E4000802F0F900F900F900F900F90DF91CF91D8
:103E50001F910F91FF90EF90DF90CF900C94D11BAA
:103E6000412F4F70602FC6010E9442270F900F9084
:103E70000F900F900F90DF91CF911F910F91FF90B6
:103E8000EF90DF90CF900C94182301112FC0FF20EA
:103E900069F10E94481C2FEF80E792E0215080409A
:103EA0009040E1F700C000000F900F900F900F902E
:103EB0000F90DF91CF911F910F91FF90EF90DF90C6
:103EC000CF900C94E426412F4F70602FC6010F90C5
:103ED0000F900F900F900F90DF91CF911F910F9146
:103EE000FF90EF90DF90CF900C9445270F900F90AC
:103EF0000F900F900F90DF91CF911F910F91FF9036
:103F0000EF90DF90CF9008951F93CF93DF9300D071
:103F100000D01F92CDB7DEB7942F4983252F5A8347
:103F20006B837C838D834C815D81452B31F02F3FEA
:103F300031F481E09F3F19F403C081E001C080E0CB
:103F4000182F117080FD24C049815A816B817C81BA
:103F50008D810E94CE24292F22952F702C3030F491
:103F60002A3048F42250223068F013C02C3061F01F
:103F70002F3051F00EC0803C28F0803E50F0815F21
:103F8000833038F011E005C093FB112710F901C010
:103F900010E0812F0F900F900F900F900F90DF91F6
:103FA000CF911F910895CF93DF9300D000D01F923F
:103FB000CDB7DEB70F900F900F900F900F90DF915D
:103FC000CF910895CF93DF9300D000D000D0CDB72C
:103FD000DEB726960FB6F894DEBF0FBECDBFDF91D9
:103FE000CF910895CF93DF93C091CA028091CB0205
:103FF000C817A1F0D0E0CE0166E070E00E94002F6B
:10400000FC01E453FD4F40815181628173818481C1
:1040100095810E94E21F2196C770E8CFDF91CF9172
:1040200008954091FC025091FD026091FE02709152
:10403000FF0280910003909101030C94E21F1F93F3
:10404000CF93DF938091010382958F7009F05CC05C
:104050008091FE02882309F457C02091CA02109172
:10406000CB02C091FC02D091FD02A091FF02B09161
:10407000000381E0CF3F09F080E0482F211709F4C9
:1040800043C0109721F0DF3F21F080E003C081E0C2
:1040900001C0842F30E080FD33C0C90166E070E0CC
:1040A0000E94002FFC01E453FD4F81818D1328C035
:1040B00080818C1325C08281811122C083819481EB
:1040C0008A1B9B0B883C9105D8F4809101038F706B
:1040D000806180930103C90166E070E00E94002FB7
:1040E000FC01EF52FD4F90819F70906190838CEFA7
:1040F00092E00E944C1CDF91CF911F910C94F21F13
:104100002F5F3F4F2770BACFDF91CF911F91089556
:104110009F92AF92BF92CF92DF92EF92FF920F9356
:104120001F93CF93DF93CDB7DEB761970FB6F894A7
:10413000DEBF0FBECDBF8C0185E0F801DE011D960C
:1041400001900D928A95E1F7F80140812181F2807A
:10415000C380D4809091FC023091FD026091FF02F7
:10416000709100036115710531F03F3F31F481E03A
:104170009F3F19F403C081E001C080E0F82FF17087
:104180009F2E80FD59C18CEFA82E82E0B82EE090C2
:10419000FE02F601E61BF70BEE2009F4EDC080915C
:1041A0000103582F507FE83CF10508F0A7C05111DA
:1041B00056C0231313C0491311C0EF2CF1100EC0C9
:1041C0008F708061809301030E941120C5010E94BD
:1041D0004C1C80910103F801858364C1C114D10492
:1041E00031F02F3F31F481E04F3F19F403C081E0FB
:1041F00001C080E080FD03C081E08F2502C080E027
:1042000090E0F82FF170EF2E80FF1FC0E091CA02FE
:104210003091CB02E31709F421C1F0E0CF0166E051
:1042200070E00E94002FDC01A453BD4F11968C91C9
:104230001197281307C08C91481304C012968C91D3
:10424000F81203C03196E770E5CFEF2CFF2009F498
:1042500029C18091010381608093010364C023130D
:1042600006C0491304C0F11002C0F801A9C04D876F
:104270002E87FF867C2DD98AC88A522F6F2D898977
:104280000E94841F8823A1F1FF2091F12091010356
:10429000822F82958F7090E0029774F08091FC02DB
:1042A0009091FD0298878F831986DB86CA862C87BA
:1042B000CE0107960E944C1C86E0F801ACEFB2E0FC
:1042C00001900D928A95E1F70E941F200E94112013
:1042D00012C0231751F14D872E87FF867C2DD98A76
:1042E000C88A522F6F2D89890E94841F81112CC08A
:1042F000C8010E944C1CEE24E394D4C05111E9CFB4
:104300007C2DD98AC88A522F6F2D89890E94D31F8C
:104310008CEF92E00E944C1C86E0F50111928A9588
:10432000E9F70E941120E12CBDC04913D4CFF11050
:10433000D2CFF8018583C8010E944C1C86E0F501AC
:1043400011928A95E9F7AEC0FF2091F22091010306
:10435000822F82958F7090E002970CF4ADCF809100
:10436000FC029091FD029A8389831B82DD82CC82BC
:104370002E83CE0101969ECFE83CF10508F04CC09B
:10438000EF2CFF2009F4B4CF231330C049132EC003
:104390002091010320FD21C0822F82958F70482F2C
:1043A00050E041155105C9F0F80125834F30510502
:1043B00041F08F5F982F9295907F822F8F70892B7D
:1043C0008583C8010E944C1C86E0F801ACEFB2E086
:1043D00001900D928A95E1F72CC086E0F801ACEFD0
:1043E000B2E001900D928A95E1F75CC04D872E876F
:1043F000FF867C2DD98AC88A522F6F2D89890E9409
:10440000841F811159CF8091010381608093010342
:10441000C8010E944C1C46C07C2DD98AC88A522FE4
:104420006F2D89890E94D31F86E0F50111928A952C
:10443000E9F70E94112036C0FF2009F459CF4D87BB
:104440002E87FF867C2DD98AC88A522F6F2D8989A5
:104450000E94841F882309F44BCF2ECF7C2DD98A4C
:10446000C88A522F6F2D89890E94CE24292F229528
:104470002F70223028F49F7039F0811105C00BC0D5
:10448000243028F49F7049F4805E883020F0C80101
:104490000E944C1C9E2CE92C05C0F8019581907F50
:1044A00099F7F9CF8E2D61960FB6F894DEBF0FBE47
:1044B000CDBFDF91CF911F910F91FF90EF90DF90D3
:1044C000CF90BF90AF909F900895CF93DF93CDB7DB
:1044D000DEB72C970FB6F894DEBF0FBECDBF4F836B
:1044E000588769877A878B879C87CE0107960E94B9
:1044F00088208823D1F09F8188852A853B85232BBE
:1045000031F08F3F31F481E09F3F19F403C081E027
:1045100001C080E080FD6FC04F81588569857A8534
:104520008B859C850E94E21F66C086E0FE0137965F
:10453000DE01119601900D928A95E1F7FF81E885E1
:104540006A857B856115710531F0EF3F31F481E0BB
:10455000FF3F19F403C081E001C080E080FD4BC043
:104560008091CB0290E09C012F5F3F4F2770332753
:104570004091CA0250E02417350709F443C0F9837B
:10458000EA837D836C8366E070E00E94002FDC018B
:10459000A453BD4F96E0FE01319601900D929A957D
:1045A000E1F72093CB020E94F21F25C090E066E065
:1045B00070E00E94002F84539D4F0E948820882322
:1045C00071F18091CA0290E066E070E00E94002FD5
:1045D000FC01E453FD4F40815181628173818481EC
:1045E00095810E94E21F8091CA0290E00196877037
:1045F00099278093CA028091CA029091CB028913B5
:10460000D5CF0DC00E94481C1092CB021092CA0256
:10461000ECEFF2E086E0DF011D928A95E9F72C9637
:104620000FB6F894DEBF0FBECDBFDF91CF910895D6
:10463000DF92EF92FF920F931F93CF93DF93FC01D2
:10464000892B09F488C0E12CF12CDD24D394EF01EF
:1046500021968491853709F460C058F4843708F0B6
:104660004EC0843008F068C08130D1F0823071F1E2
:1046700072C0883709F45BC050F4863709F453C020
:10468000873709F068C08E2D0E94A42552C09CE790
:10469000980F903708F05FC08F770E94D11B4EC0F3
:1046A0008F010E5F1F4FFE01849190E2980F9830AA
:1046B00050F48770FD2D01C0FF0F8A95EAF78F2F08
:1046C0000E94AA2515C00E94DB1A14C08F010E5F3C
:1046D0001F4FFE01849190E2980F983068F4877024
:1046E000FD2D01C0FF0F8A95EAF78F2F0E94B0259C
:1046F0000E94D125E80122C00E94D11BFBCFCF012F
:104700000296FE01C491CC2361F0EFE9FFE03197FE
:10471000F1F700C00000C150F6CFCF010296FE01B4
:10472000F490EC010BC00E949425E82E07C00E9473
:10473000A7250E94D12502C00E94DB1A8F2D882355
:1047400041F0EFE9FFE03197F1F700C00000815040
:10475000F6CFFE017CCFDF91CF911F910F91FF909B
:10476000EF90DF90089560938203709383038093AA
:104770008403909385030C941F2608956093860309
:104780007093870380938803909389030C941E266B
:104790000F931F9300918603109187032091880344
:1047A00030918903602B712B822B932B60938603AE
:1047B0007093870380938803909389031F910F91CF
:1047C0000C941E260F931F9300918603109187036C
:1047D00020918803309189036023712382239323DE
:1047E0006093860370938703809388039093890373
:1047F0001F910F910C941E260F931F930091860317
:1048000010918703209188033091890360277127D5
:10481000822793276093860370938703809388038E
:10482000909389031F910F910C941E2660E070E015
:10483000CB010C94B3230F931F9341E050E060E051
:1048400070E08A019B0104C0000F111F221F331F5B
:104850008A95D2F7C901B8011F910F910C94B32327
:104860000F931F9341E050E060E070E004C0440FFC
:10487000551F661F771F8A95D2F78091820390910A
:104880008303A0918403B09185038A019B01082BC7
:10489000192B2A2B3B2BC901B8011F910F910C94A6
:1048A000B3230F931F9341E050E060E070E004C039
:1048B000440F551F661F771F8A95D2F74095509574
:1048C000609570958091820390918303A0918403F9
:1048D000B09185038A019B01082319232A233B23D6
:1048E000C901B8011F910F910C94B3230F931F932B
:1048F00041E050E060E070E004C0440F551F661FC7
:10490000771F8A95D2F78091820390918303A091BB
:104910008403B09185038A019B01082719272A2760
:104920003B27C901B8011F910F910C94B3230F933A
:104930001F9300918203109183032091840330918F
:104940008503602B712B822B932B1F910F910C945D
:10495000B3230F931F93009182031091830320913F
:1049600084033091850360237123822393231F9155
:104970000F910C94B3230F931F9300918203109116
:104980008303209184033091850360277127822758
:1049900093271F910F910C94B32308958F929F92A8
:1049A000AF92BF92DF92EF92FF920F931F93CF933C
:1049B000DF9300D000D01F92CDB7DEB76B837C832E
:1049C0008D838A018C819D81892B31F01F3F31F4C9
:1049D00081E04F3F19F403C081E001C080E080FF17
:1049E00003C080E090E054C08B81882309F43DC06F
:1049F0008090820390908303A0908403B0908503FD
:104A00008091860390918703A0918803B0918903D8
:104A1000882A992AAA2ABB2A2FE1E22EF12CD50155
:104A2000C4010E2C04C0B695A795979587950A9456
:104A3000D2F780FD06C081E0E81AF10880F7D12C9A
:104A400007C0DE2CB8018E2D0E941527019799F31F
:104A5000E12FF0E093E0EE0FFF1F9A95E1F7EE5F94
:104A6000FC4FE00FF11DD0820CC0E12FF0E083E09D
:104A7000EE0FFF1F8A95E1F7EE5FFC4FE00FF11D8F
:104A8000D08009831A8369817A818D2D0E94152730
:104A90000F900F900F900F900F90DF91CF911F917B
:104AA0000F91FF90EF90DF90BF90AF909F908F900D
:104AB00008952091150130911601F90132969FEF6A
:104AC00040E05191851789F09F3F19F4511101C0C1
:104AD000942F4F5F4630A9F79F3F39F0F901E90F56
:104AE000F11D97FDFA95828308950895E0911501CF
:104AF000F09116019F012A5F3F4F9281891301C0F7
:104B000012823196E217F307C1F7089581E090E031
:104B1000E0911501F0911601E80FF91F108201963E
:104B200088309105A9F70895809194030895909194
:104B30009403892B80939403089580959091940316
:104B40008923809394030895809394030895109289
:104B50009403089590919303892B80939303089570
:104B600080959091930389238093930308951092E5
:104B70009303089580938A03089510928A030895F9
:104B80008091150190911601FC0131969C01285FDE
:104B90003F4F80E0919191118F5FE217F307D1F7BA
:104BA0000895E0911501F09116018091940380839E
:104BB000E0911501F0911601908180919303892B6A
:104BC000808380918A03882361F0E0911501F09140
:104BD00016019081892B80830E94C025811110923B
:104BE0008A0380911501909116010C94D41890932A
:104BF00055018093540108958295982F9373292F1E
:104C0000220F220F982F9C7C96959695922B892F98
:104C10008575880F9A7A9695892B08950895CF9374
:104C2000DF9300D000D01F92CDB7DEB70F900F906A
:104C30000F900F900F90DF91CF91089508950895F0
:104C40000C94471A80E008958091AA03843021F1E2
:104C50001092960320E488E190E00FB6F894A895AE
:104C6000809360000FBE2093600083B7817F8460D3
:104C700083BF83B7816083BF7894889583B78E7F25
:104C800083BF0FB6F894A8958091600088618093E7
:104C90006000109260000FBE0895CF930E94931A97
:104CA0000E94F60A0E94941AC0E08C2F0E94F80A13
:104CB000811104C0CF5FC031C1F701C081E0CF9145
:104CC00008950E94491A0C94481C1F920F920FB627
:104CD0000F9211248F939F93AF93BF93809196036C
:104CE000811113C08091970390919803A09199032B
:104CF000B0919A034196A11DB11D809397039093A3
:104D00009803A0939903B0939A03BF91AF919F9199
:104D10008F910F900FBE0F901F90189582E084BD69
:104D200093E095BD9AEF97BD80936E0008952FB7DD
:104D3000F8948091970390919803A0919903B09172
:104D40009A032FBF08952FB7F8946091970370913D
:104D500098038091990390919A032FBF08959C0125
:104D60004FB7F8948091970390919803A09199037D
:104D7000B0919A034FBF821B930B089578941F92B2
:104D80000F920FB60F9211248F939F93AF93BF93FF
:104D90008091970390919803A0919903B0919A0301
:104DA0000196A11DB11D8093970390939803A09342
:104DB0009903B0939A03BF91AF919F918F910F90F8
:104DC0000FBE0F901F9018950E949A17F89487E7CE
:104DD00097E7909301088093000887E090EBDC014F
:104DE0008093B3039093B403A093B503B093B60339
:104DF0009CE088E10FB6F894A895809360000FBE00
:104E000090936000FFCFE92FF0E093E0EE0FFF1FDB
:104E10009A95E1F7E80FF11DE855FF4F8491982F1F
:104E200092959F708F7097700895CF93C82FCB0184
:104E30000E940327292F30E054E0220F331F5A9598
:104E4000E1F7282B203831051CF080E090E018C0F5
:104E5000EC2FF0E023E0EE0FFF1F2A95E1F79770AB
:104E6000E90FF11D34E0EE0FFF1F3A95E1F78F7067
:104E7000E80FF11DEE0FFF1FE050F8498591949166
:104E8000CF91089580E090E00895089580919D036A
:104E900080FF0CC080911A0190E065E070E00E94F4
:104EA000002F95958795959587952EC081FF0AC00F
:104EB00080911A0190E065E070E00E94002F9595C6
:104EC000879522C082FF08C080911A0190E065E0BA
:104ED00070E00E94002F18C020919E032223D9F079
:104EE00030911901231780F780911A0190E065E055
:104EF00070E00E94002F622F70E00E94002F632F4D
:104F000070E00E94112FCB018038910538F4009792
:104F100039F481E005C085E090E008958FE70895B9
:104F2000089580919D0380FF08C06091180170E092
:104F3000759567957595679523C081FF06C060914B
:104F4000180170E0759567951BC082FF04C06091E1
:104F5000180170E012C060919E036623A9F02091B1
:104F600017016217A0F78091180170E090E00E948D
:104F7000002F622F70E00E94112F6038710540F4FD
:104F80006115710519F406C061E070E0862F08957F
:104F90008FE7089581E00895803F21F40E9446271D
:104FA000819504C0813F29F40E9446278093A10384
:104FB0000895823F21F40E944627819504C0833FD3
:104FC00029F40E9446278093A0030895893F19F48D
:104FD0000E94912705C08A3F31F40E949127819554
:104FE0008093A20308958B3F21F40E94912781951D
:104FF00004C08C3F29F40E9491278093A303089555
:10500000843F21F480919F03816017C0853F21F484
:1050100080919F03826011C0863F21F480919F039D
:1050200084600BC0873F21F480919F03886005C096
:10503000883F31F480919F03806180939F0308959E
:105040008D3F21F480919D0381600BC08E3F21F440
:1050500080919D03826005C08F3F29F480919D035C
:10506000846080939D030895803F39F48091A1036B
:1050700087FF6CC01092A10369C0813F29F4809121
:10508000A1031816BCF362C09091A003823F29F4DB
:1050900097FF5CC01092A00359C0833F19F4191602
:1050A000CCF354C0893F41F48091A20318160CF050
:1050B0004DC01092A2034AC08A3F29F48091A203F6
:1050C00087FF44C0F6CF8B3F39F48091A30387FF5D
:1050D0003DC01092A3033AC08C3F29F48091A303F2
:1050E0001816BCF333C0843F21F480919F038E7F58
:1050F00017C0853F21F480919F038D7F11C0863FAB
:1051000021F480919F038B7F0BC0873F21F4809116
:105110009F03877F05C0883F31F480919F038F7E76
:1051200080939F0313C08D3F21F480919D038E7F58
:105130000BC08E3F21F480919D038D7F05C08F3F72
:1051400029F480919D038B7F80939D038091A00320
:1051500081110EC08091A10381110AC08091A20328
:10516000811106C08091A303811102C010929E0399
:1051700008958091950383FF7EC08CEF95E00E9497
:10518000450680919F031F928F9387EF95E09F9331
:105190008F930E94DE0685EF95E00E944506809180
:1051A000A003282F082E000C330B3F938F9382EF20
:1051B00095E09F938F930E94DE0680EF95E00E941A
:1051C00045068091A103282F082E000C330B3F9336
:1051D0008F938DEE95E09F938F930E94DE068BEE6A
:1051E00095E00E9445068091A203282F082E000C0E
:1051F000330B3F938F9388EE95E09F938F930E949C
:10520000DE0686EE95E00E9445068091A303282FD6
:10521000082E000C330B3F938F9383EE95E09F9302
:105220008F930E94DE0680EE95E00E9445068091F5
:105230009E031F928F938DED95E09F938F930E9415
:10524000DE068BED95E00E94450680919D031F923E
:105250008F9388ED95E09F938F930E94DE0685EDF6
:1052600095E00E9445068DB79EB74C960FB6F89410
:105270009EBF0FBE8DBF8FE993E00E941D190E9453
:10528000972690939C0380939B0308951F93CF933D
:10529000DF9380919B0390919C030E94AF26FC01B9
:1052A00020919E03222321F080911B0190E007C0F2
:1052B00080911C0190E06AE070E00E94002FE817E6
:1052C000F90708F485C08091A003C091A103D09193
:1052D000A2031091A303811107C0C11175C0D111A0
:1052E00073C0111171C074C02F3F19F02F5F20934C
:1052F0009E03181624F40E9446278093A0038091F1
:10530000A00387FF05C00E94462781958093A003D4
:105310001C1624F40E9446278093A1038091A103C8
:1053200087FF05C00E94462781958093A103609165
:10533000A003662331F1C091A103CC2311F1062E05
:10534000000C770B880B990B0E94FF2D23E333E3AE
:1053500043E35FE30E94632E0E94C72D6093A00386
:105360006C2FCC0F770B880B990B0E94FF2D23E33A
:1053700033E343E35FE30E94632E0E94C72D6093F3
:10538000A1031D1624F40E9491278093A20380910B
:10539000A20387FF05C00E94912781958093A203F5
:1053A000111624F40E9491278093A3038091A303F4
:1053B00087FF05C00E94912781958093A303DF9109
:1053C000CF911F910C94B9282F3F09F08FCFA0CF18
:1053D000DF91CF911F910895EFE9F3E085E0DF01C0
:1053E0001D928A95E9F710929E0310929D030895ED
:1053F00080919F0308958FE198E00E9445061F92D7
:1054000081E08F931F9285E08F9381ED97E09F93CA
:105410008F930E94DE060F900F900F900F900F90C9
:105420000F9008958330E9F128F4813061F08230E3
:1054300009F10895853009F462C008F449C0863046
:1054400009F474C0089580911C01262F30E0280FC4
:10545000311D2F3F310524F4680F60931C0103C0F8
:105460008FEF80931C0180911C011F928F938AE023
:1054700097E072C080911B01262F30E0280F311D6C
:105480002F3F310524F4680F60931B0103C08FEF99
:1054900080931B0180911B011F928F9388EF96E0F0
:1054A0005BC080911A01262F30E0280F311D2F3F5D
:1054B000310524F4680F60931A0103C08FEF8093C5
:1054C0001A0180911A011F928F9385EE96E044C0D5
:1054D00080911901262F30E0280F311D2F3F310513
:1054E00024F4680F6093190103C08FEF80931901B2
:1054F000809119011F928F9380ED96E02DC08091CD
:105500001801262F30E0280F311D2F3F310524F4DC
:10551000680F6093180103C08FEF8093180180918A
:1055200018011F928F9387EB96E016C080911701A8
:10553000262F30E0280F311D2F3F310524F4680F4E
:105540006093170103C08FEF8093170180911701BB
:105550001F928F938CE996E09F938F930E94DE06B3
:105560000F900F900F900F900895833081F128F4E1
:10557000813059F08230D1F00895853009F449C066
:10558000B8F1863009F456C0089580911C0168175F
:1055900020F4861B80931C0102C010921C01809194
:1055A0001C011F928F938DE896E054C080911B01DF
:1055B000681720F4861B80931B0102C010921B0108
:1055C00080911B011F928F938BE796E043C08091DF
:1055D0001A01681720F4861B80931A0102C01092EA
:1055E0001A0180911A011F928F9388E696E032C0CB
:1055F00080911901681720F4861B8093190102C05D
:1056000010921901809119011F928F9383E596E002
:1056100021C080911801681720F4861B809318011F
:1056200002C010921801809118011F928F938AE393
:1056300096E010C080911701681720F4861B8093B4
:10564000170102C010921701809117011F928F93CA
:105650008FE196E09F938F930E94DE060F900F904C
:105660000F900F900895CF93C82F1F928F9384E2CD
:1056700099E09F938F930E94DE0681E090E0A0E086
:10568000B0E0BC01CD0104C0660F771F881F991FD1
:10569000CA95D2F70E94BE230F900F900F900F90E3
:1056A000CF910C94481CCF93873288F58E3108F047
:1056B0000BC18E3009F487C0D8F4873009F460C07C
:1056C0008B3009F44FC0863009F002C180919503F8
:1056D000817F8E7F8093950389E299E00E94450641
:1056E00089ED9BE00E94450681E08093A50346C0BA
:1056F000863109F4B0C020F4803109F47AC0E8C0E2
:10570000893109F491C08B3109F449C0E1C0883373
:1057100049F150F4893209F4D5C0853309F4D2C077
:10572000873209F0D5C0CEC0833409F4CBC028F449
:105730008A3308F4CDC08953C8C0883409F0C8C082
:105740000E94481C88EC9BE00E9445062FEF83EDE9
:1057500090E3215080409040E1F700C000000E949B
:10576000E4260CC080E599E041C08FEA9BE00E94EE
:10577000450680919503816080939503C1E0ADC09B
:1057800080919503C82FC17080FFEFCF8BEB9BE01A
:105790000E94450680919503817F8E7F3FC0909146
:1057A000950391FBCC27C0F981E0C827892FC0FB66
:1057B00081F980939503CC2319F082EA9BE029C0FC
:1057C00084E99BE013C09091950392FBCC27C0F92C
:1057D00081E0C827892FC0FB82F980939503CC23F1
:1057E00019F085E89BE015C085E79BE00E9445061F
:1057F000C5CF9091950393FBCC27C0F981E0C827D2
:10580000892FC0FB83F980939503CC2351F089E65F
:105810009BE00E94450680919503816080939503EB
:105820005CC08CE59BE0E2CF8DE49BE00E944506E6
:105830008AE29BE00E94450685EE9AE00E944506BA
:105840008FEB9AE00E9445068AE79AE00E9445069F
:105850008EE49AE0CBCF80E49AE00E9445060E9455
:10586000C8181F928F9386E29AE09F938F930E94AD
:10587000DE06809114011F928F938FE09AE09F9330
:105880008F930E94DE068091B2021F928F938CEF5D
:1058900099E09F938F930E94DE060E94A3269F9318
:1058A0008F937F936F9385EE99E09F938F930E94E0
:1058B000DE068DB79EB742960FB6F8949EBF0FBE18
:1058C0008DBF5CCF80E001C08D510E94332B56CF3D
:1058D00083EE99E00E944506C0E08C2FCF91089599
:1058E00080E008950C94702CCF93C82F8091A5036D
:1058F000813069F020F0823009F449C040C167E08E
:105900008FE00E944B1A882309F43FC106C067E06C
:105910008FE00E944B1A882361F08C2F0E94722C1A
:10592000811104C08C2F0E94532B2FC081E090E086
:105930002CC08C2F0E94702C811126C0C431E1F044
:1059400070F4CB3081F0C031D1F40E94FB298CE19E
:1059500099E00E94450682E08093A50315C0C932F4
:1059600059F0C83361F489E299E00E94450680E26B
:1059700099E00E94450608C01092A50304C18AE17F
:1059800099E00E944506FFC081E08170FEC0C432EC
:1059900028F5CE3108F0C1C0CB30A1F1D0F4C7302A
:1059A00009F0D3C08EE180931C0182E380931B0138
:1059B0008AE080931A0184E18093190188E0809342
:1059C000180188E28093170180EC97E00E94450659
:1059D000BFC0C33149F1C431C1F0B7C0CB3409F401
:1059E000A9C028F4C93289F0C83361F0AEC0C1350E
:1059F00009F49EC0C23509F499C0CE3409F0A5C09F
:105A00006AE09EC00E94FB29A3C08091A403882362
:105A100019F01092A4039CC08DEC97E00E944506FB
:105A200081E08093A503B1C087EA97E00E94450614
:105A300085E997E00E94450680911C011F928F9393
:105A400082E997E09F938F930E94DE0680E997E0BA
:105A50000E9445068EE797E00E94450680911B0153
:105A60001F928F938BE797E09F938F930E94DE06A0
:105A700089E797E00E9445068AE697E00E9445067E
:105A800080911A011F928F9387E697E09F938F93DF
:105A90000E94DE0685E697E00E94450684E597E0D1
:105AA0000E944506809119011F928F9381E597E02E
:105AB0009F938F930E94DE068FE497E00E94450635
:105AC0008AE397E00E944506809118011F928F9308
:105AD00087E397E09F938F930E94DE0685E397E02C
:105AE0000E9445068EE197E00E94450680911701CD
:105AF0001F928F938BE197E09F938F930E94DE0616
:105B000089E197E00E9445068DB79EB748960FB68B
:105B1000F8949EBF0FBE8DBF1BC0CE51EC2FF0E09E
:105B2000E75BFE4F80818093A40312C061E003C055
:105B300061E006C06AE08091A4030E94122A08C0B6
:105B40008091A4030E94B52A03C08EEB97E013C096
:105B50008091A403882369F01F928F9388EB97E0CC
:105B60009F938F930E94DE060F900F900F900F90DF
:105B700004C085EB97E00E94450681E006C01092C4
:105B8000A50380E002C080E000CFCF9108950E947D
:105B9000CE2D6894B1110C945D2E08950E94422E72
:105BA00088F09F5798F0B92F9927B751B0F0E1F0DE
:105BB000660F771F881F991F1AF0BA95C9F714C08E
:105BC000B13091F00E945C2EB1E008950C945C2EEF
:105BD000672F782F8827B85F39F0B93FCCF38695C7
:105BE00077956795B395D9F73EF490958095709524
:105BF00061957F4F8F4F9F4F0895E89409C097FBA1
:105C00003EF490958095709561957F4F8F4F9F4F93
:105C10009923A9F0F92F96E9BB279395F6958795D7
:105C200077956795B795F111F8CFFAF4BB0F11F49A
:105C300060FF1BC06F5F7F4F8F4F9F4F16C0882341
:105C400011F096E911C0772321F09EE8872F762F77
:105C500005C0662371F096E8862F70E060E02AF0B8
:105C60009A95660F771F881FDAF7880F96958795A4
:105C700097F9089557FD9058440F551F59F05F3F0D
:105C800071F04795880F97FB991F61F09F3F79F05E
:105C900087950895121613061406551FF2CF4695E0
:105CA000F1DF08C0161617061806991FF1CF869562
:105CB0007105610508940895E894BB276627772746
:105CC000CB0197F908950E94752E0C94EF2E0E9437
:105CD000E12E38F00E94E82E20F0952311F00C946C
:105CE000D82E0C94DE2E0C945D2E0E943A2E78F362
:105CF0009923C9F35523B9F3950F50E0551FAA27EF
:105D0000EE27FF27BB2700240894679520F4E20FB5
:105D1000F31FB41F0A1E220F331F441FAA1F6695CC
:105D2000A9F7779530F4F30FB41F0A1E121E08F47A
:105D30006395330F441FAA1F221F769599F7879505
:105D400020F4B40F0A1E121E631F440FAA1F221F45
:105D5000331F8695A9F7862F712D602D11249F572B
:105D600050409AF0F1F088234AF0EE0FFF1FBB1F5E
:105D7000661F771F881F91505040A9F79E3F51051D
:105D800080F00C94D82E0C945D2E5F3FE4F3983E87
:105D9000D4F3869577956795B795F795E7959F5FC7
:105DA000C1F7FE2B880F911D9695879597F9089559
:105DB00097F99F6780E870E060E008959FEF80ECBE
:105DC000089500240A941616170618060906089561
:105DD00000240A9412161306140605060895092EC7
:105DE0000394000C11F4882352F0BB0F40F4BF2B36
:105DF00011F460FF04C06F5F7F4F8F4F9F4F089576
:105E00000024552704C0080E591F880F991F0097BA
:105E100029F076956795B8F37105B9F7802D952F20
:105E2000089597FB072E16F4009407D077FD09D04C
:105E30000E942B2F07FC05D03EF4909581959F4F33
:105E40000895709561957F4F0895EE0FFF1F05909F
:105E5000F491E02D0994AA1BBB1B51E107C0AA1FB6
:105E6000BB1FA617B70710F0A61BB70B881F991FFB
:105E70005A95A9F780959095BC01CD010895F894A5
:025E8000FFCF52
:105E8200FFFF0305A9010000FF931035110611CA97
:105E920010961001018B032808140A321E0000100C
:105EA20007B514000069FFFF37414E5349004953BB
:105EB2004F004A4953003F3F3F00407F224105C205
:105EC20004A0044C0465047E0401020304050607D1
:045ED20008090000BB
:106800008800EA44E944E244040005000600070069
:10681000080009000A000B000C000D000E000F001C
:1068200010001100120013001400150016001700CC
:10683000180019001A001B001C001D001E001F007C
:10684000200021002200230024002500260027002C
:10685000280029002A002B002C002D002E002F00DC
:10686000300031A132003300340035A1360037004A
:10687000380082003A003B003C003D003E003F00F3
:1068800040004100420043004400450046004700EC
:10689000480049004A004B004C004D004E004F009C
:1068A00050005100520053002E0054005500560075
:1068B000580059005A005B005C005D005E005F00FC
:1068C0006000610062006300640000005700850002
:1068D000CD440000000000000000000000000000A7
:1068E000000000000000A520890087008A008B00BE
:1068F000E000E100E200E300E400E500E600000063
:106900000100010001000100EA4401000100E2442D
:106910000100010001000100460001004A004B0097
:10692000010001004700480001000100E9440100A6
:106930000100010001000100010001003A003B00DC
:106940003C003D003E003F0040004100420043004B
:10695000010035004C0001000100440045005200D8
:1069600049000100010050004F0029004D004E0079
:1069700051000100010001000100010001000100BF
:1069800001000100010001000100010001000100FF
:1069900001000100010001000100010001004D00A3
:1069A0004A004E004B0001000100010001000100FF
:1069B00001000100010001000100010001000100CF
:1069C00001000100010001000100000001000100C0
:1069D00001000000000000000000000000000000B6
:1069E000000000000000010049000100010001005A
:1069F0000100010001000100010001000100000090
:00000001FF
